:10800000FEDF07EA000000000000000000000000A2
:108010000000000000000000000000000000000060
:108020000000000000000000000000000000000050
:108030000000000000000000000000000000000040
:108040000000000000000000000000000000000030
:02000004001FDB
:020000040020DA
:1000000002D3A0E39F0000EBFEFFFFEA001080E5B3
:100010001EFF2FE1B010C0E11EFF2FE10010C0E570
:100020001EFF2FE1000090E51EFF2FE10E00A0E172
:100030001EFF2FE110FF2FE11EFF2FE108402DE9E9
:1000400008009FE5F6FFFFEB0840BDE81EFF2FE12B
:100050005450212008402DE91C009FE5F0FFFFEBE4
:10006000010010E3FBFFFF0A10009FE5ECFFFFEB30
:10007000FF0000E20840BDE81EFF2FE154502120A0
:100080004050212010402DE90040A0E11C009FE5D8
:10009000E3FFFFEB200010E3FBFFFF0A10009FE5EA
:1000A0000410A0E1D8FFFFEB1040BDE81EFF2FE1D8
:1000B000545021204050212008402DE910009FE598
:1000C000D7FFFFEB010C10E3FBFFFF1A0840BDE870
:1000D0001EFF2FE15450212038402DE90050A0E1AF
:1000E0002040A0E3044044E23534A0E10F3003E2B5
:1000F000090053E33700838230008392E0FFFFEB77
:10010000000054E3F6FFFF1A2000A0E33840BDE8EA
:10011000DBFFFFEA08402DE9EEFFFFEB0D00A0E357
:10012000D7FFFFEB0A00A0E30840BDE8D4FFFFEAD9
:1001300010402DE9D8009FE50110A0E3B2FFFFEBCE
:10014000D0009FE50010A0E3AFFFFFEBC8009FE5E4
:100150000010A0E3ACFFFFEBC0009FE50310A0E39D
:10016000A9FFFFEBB8009FE50010A0E3A6FFFFEB9F
:10017000A0009FE50010A0E3A3FFFFEBA4009FE514
:10018000C610A0E3A0FFFFEB9C109FE59C009FE53D
:100190009DFFFFEB98009FE5A1FFFFEB3F1AC0E337
:1001A000121A81E388009FE597FFFFEB84009FE52B
:1001B0000010A0E394FFFFEB0040A0E30400A0E1E7
:1001C000014084E29BFFFFEB960054E3FAFFFF1A25
:1001D00064009FE50319A0E38BFFFFEB0040A0E361
:1001E0000400A0E1014084E292FFFFEB960054E39B
:1001F000FAFFFF1A40009FE50010A0E382FFFFEB2B
:1002000014009FE50310A0E37FFFFFEB1040BDE863
:100210001EFF2FE104502120445021206050212056
:100220004C50212050502120485021200E01000028
:1002300068502120040020209400202098002020D5
:1002400010402DE91C409FE5F918A0E30400A0E14F
:100250006DFFFFEB0400A0E10C109FE56AFFFFEBD0
:100260001040BDE81EFF2FE108B400200002F90095
:1002700008402DE908009FE569FFFFEB0840BDE855
:100280001EFF2FE120B40020F04F2DE90CD04DE2ED
:10029000A6FFFFEBD8019FE59DFFFFEB62FFFFEBA1
:1002A0009BFFFFEB0209A0E399FFFFEBE3FFFFEBEE
:1002B000EEFFFFEBBC919FE50239A0E30080A0E3D5
:1002C00004308DE5B0719FE50860A0E101B0A0E3C6
:1002D0000050A0E109A0A0E1824089E2E3FFFFEB2A
:1002E000000065E0070050E11700008A52FFFFEBB5
:1002F000010010E3F8FFFF0A55FFFFEB0600C9E716
:10030000DAFFFFEB000056E30050A0E11300001AF3
:100310000030DAE5040053E34100000A0030D9E57B
:10032000010053E30380A0010860A001EAFFFF0A77
:100330001500A0E352FFFFEBCCFFFFEB000065E0F0
:10034000070050E10060A0E3E7FFFF9A1500A0E37B
:100350003D5885E24AFFFFEB095C85E2E2FFFFEAD8
:10036000010056E30800000AEBFFFF3A020056E3E3
:100370002300000A830056E30900000A0630DAE78A
:10038000016086E2038088E0D3FFFFEA0130DAE50E
:100390000B0053E10B8088000260A003E3FFFF1A0B
:1003A000CDFFFFEA8330DAE5FF8008E2080053E181
:1003B00000308DE5DDFFFF1AC0809FE504309DE52C
:1003C0000110F8E50300A0E1016083E212FFFFEBFA
:1003D000040058E10630A0E1F8FFFF1A0600A0E390
:1003E00027FFFFEB04309DE501B08BE2803083E214
:1003F00004308DE5FFB00BE200809DE50060A0E3D6
:10040000B5FFFFEA0120DAE50230DAE5FF2062E21B
:10041000020053E1038088000360A003C3FFFF1ABA
:10042000ADFFFFEA0600A0E315FFFFEB0600A0E129
:10043000016086E236FFFFEB1E0056E3FAFFFF1A6B
:100440003C009FE532FFFFEB38009FE530FFFFEBFC
:1004500034009FE52EFFFFEB16FFFFEB0209A0E340
:10046000F3FEFFEB0000A0E30CD08DE2F04FBDE8FF
:100470001EFF2FE17856341290042000FF083D0043
:10048000920420001111111122222222333333331E
:040000030000800079
:00000001FF
